:100000000C9447060C947F060C947F060C947F0694
:100010000C947F060C947F060C947F060C947F064C
:100020000C947F060C947F060C94B72B0C94892CAF
:100030000C94ED250C947F060C947F060C947F069F
:100040000C947F060C94111E0C947F060C947F0672
:100050000C94F01E0C9475260C947F060C947F066D
:100060000C947F060C947F060C947F060C947F06FC
:100070000C947F060C947F060C947F060C947F06EC
:100080000C947F060C947F060C947F060C947F06DC
:100090000C947F060C947F060C947F060C947F06CC
:1000A0000C947F060C947F060C947F06590A590A1B
:1000B000850A850AED0A0B0B230C230C160BAF0BDC
:1000C000C00BC00B661D681D6D1D701D731D761D58
:1000D000791DF62C1D2D152E1D2D152E692D8C2DFF
:1000E000152EE32DF22D29001E001F0020002100F7
:1000F0002200230024002500260027002D002E00CA
:1001000035002A0049002B0014001A0008001500D1
:1001100017001C0018000C00120013002F00300004
:1001200031004C00000039000400160007000900EF
:100130000A000B000D000E000F00330034002800F1
:10014000000000000000E10064001D001B0006002C
:100150001900050011001000360037003800E500D6
:10016000015152000000E000E300E2002C002C00EE
:10017000E6000151E400500051004F000000000073
:1001800000000000000035003A003B003C003D004C
:100190003E003F0040004100420043004400450053
:1001A0002A002A00490001000100010001000100AD
:1001B000010001000100010001000100AA00A900E6
:1001C000A8004C000000005C0100010001000100DB
:1001D0000100010001000100010001000100010017
:1001E000000000000000010001000100010001000A
:1001F0000100010001000100C25CC15CA600010019
:1002000001004B000000010001000100010001009D
:100210000100010001004A004E004D0000000000F6
:1002200000000000000044454255473A20646973CD
:1002300061626C65642E0A0044454255473A206568
:100240006E61626C65642E0A000A00253032580027
:100250006C65645F7461736B3A20004F6E65736800
:100260006F743A206163746976653A2025640A00E8
:100270000A002530313662003A200025303258001D
:100280000A722F63203031323334353637383941F2
:1002900042434445460A00290A002575002F0025DF
:1002A00075005D28002564002000256400200025DD
:1002B000640020002564007C0025303258006D6FFA
:1002C0007573656B6579205B62746E7C782079202C
:1002D0007620685D287265702F61636C293A205B17
:1002E000006261636B6C6967687420627265617437
:1002F00068696E672064697361626C650A00626197
:10030000636B6C6967687420627265617468696E9A
:100310006720656E61626C650A006261636B6C697F
:1003200067687420627265617468696E6720746FB3
:1003300067676C653A2025750A006261636B6C69BA
:1003400067687420737465703A2025750A006261CD
:10035000636B6C696768742064697361626C650AB9
:10036000006261636B6C6967687420656E61626CC2
:10037000650A006261636B6C6967687420746F67FB
:10038000676C653A2025750A006261636B6C69676A
:1003900068742064656372656173653A2025750A27
:1003A000006261636B6C6967687420696E63726573
:1003B0006173653A2025750A000000000000000006
:1003C0000000000001010203040506080A0C0F11D9
:1003D00014181C2024292E33393F464C535B626A83
:1003E0007179818A929AA2AAB2B9C1C8CFD5DCE14B
:1003F000E7EBF0F4F7FAFCFDFEFFFEFDFCFAF7F484
:10040000F0EBE7E1DCD5CFC8C1B9B2AAA29A928AD3
:100410008179716A625B534C463F39332E2924201F
:100420001C1814110F0C0A08060504030201010030
:10043000000000000000000000313A0964656C61B2
:1004400079282A31306D73293A2025750A323A0904
:10045000696E74657276616C286D73293A20257512
:100460000A333A096D61785F73706565643A2025D7
:10047000750A343A0974696D655F746F5F6D6178F0
:100480003A2025750A353A09776865656C5F6D61B4
:10049000785F73706565643A2025750A363A097786
:1004A0006865656C5F74696D655F746F5F6D6178B9
:1004B0003A2025750A00703A097072696E742076C8
:1004C000616C7565730A643A0973657420646566C6
:1004D00061756C74730A75703A092B310A646E3A4F
:1004E000092D310A6C743A092B31300A72743A09B9
:1004F0002D31300A4553432F713A09717569740AD9
:100500000A7370656564203D2064656C7461202AFF
:10051000206D61785F7370656564202A202872659C
:1005200070656174202F2074696D655F746F5F6DF5
:100530006178290A77686572652064656C74613A30
:1005400020637572736F723D25642C207768656532
:100550006C3D25640A53656520687474703A2F2FCA
:10056000656E2E77696B6970656469612E6F72675D
:100570002F77696B692F4D6F7573655F6B65797345
:100580000A004D3E20004D25753A25733E20003F60
:100590000A003D2025750A003F0A00646566617502
:1005A0006C74730A0025750A003F0A000A092D20A1
:1005B00056616C756573202D0A00710A000A092DB9
:1005C000204D6F7573656B6579202D0A003F0043E0
:1005D0003E20004C25640A000A092D2053746174E2
:1005E0007573202D0A686F73745F6B6579626F6134
:1005F00072645F6C65647328293A20253032580A8A
:100600006B6579626F6172645F70726F746F636F34
:100610006C3A20253032580A6B6579626F617264DA
:100620005F69646C653A20253032580A74696D65DB
:10063000725F72656164333228293A202530386C44
:10064000580A000A092D2056657273696F6E202DB5
:100650000A5649443A2030784645454428414D4A97
:100660004B6579626F61726429205049443A2030A9
:10067000784244363628414D4A363629205645526E
:100680003A203078303030310A4255494C443A20D3
:1006900020284665622032372032303232290A4F14
:1006A0005054494F4E533A204C554641204D4F55DA
:1006B00053454B45592045585452414B45592043C9
:1006C0004F4E534F4C4520434F4D4D414E442034E7
:1006D0003039360A4743433A20352E342E302041F4
:1006E00056522D4C4942433A20322E302E30204172
:1006F00056525F415243483A20617672350A000AE9
:10070000092D20436F6E736F6C65202D0A4553438E
:100710002F713A09717569740A6D3A096D6F7573B5
:10072000656B65790A000A092D204D6167696320B0
:100730002D0A443A094465627567204D65737361FB
:10074000676520546F67676C650A583A094D617494
:10075000726978204465627567204D6F6465205426
:100760006F67676C65202D2053686F77206B657904
:100770007072657373657320696E206D6174726940
:100780007820677269640A4B3A094B6579626F6138
:10079000726420446562756720546F67676C6520DA
:1007A0002D2053686F77206B6579707265737320A5
:1007B0007265706F72740A4D3A09446562756720FC
:1007C0004D6F75736520546F67676C650A563A09FB
:1007D00056657273696F6E0A533A09537461747582
:1007E000730A433A09416374697661746520436F03
:1007F0006E736F6C65204D6F64650A46312D46310E
:10080000303A0953776974636820746F204C6179BA
:10081000657220302D392028463130203D204C3063
:10082000290A302D393A0953776974636820746F47
:10083000204C6179657220302D390A475241564566
:100840003A0953776974636820746F204C61796545
:100850007220302028616C7465726E617465290A9B
:10086000423A094A756D7020746F20426F6F746C44
:100870006F616465720A4553433A094A756D702089
:10088000746F20426F6F746C6F61646572202861B1
:100890006C7465726E617465290A453A0950726913
:1008A0006E7420454550524F4D2053657474696EE7
:1008B00067730A4253504143453A09436C6561727C
:1008C00020454550524F4D0A006261636B6C696769
:1008D00068745F636F6E6669672E7261773A202570
:1008E0003032580A2E656E61626C653A2025750AB1
:1008F0002E6C6576656C3A2025750A006B65796DFE
:1009000061705F636F6E6669672E7261773A20254A
:100910003032580A2E737761705F636F6E74726F36
:100920006C5F636170736C6F636B3A2025750A2E80
:10093000636170736C6F636B5F746F5F636F6E7412
:10094000726F6C3A2025750A2E737761705F6C6345
:10095000746C5F6C6775693A2025750A2E73776130
:10096000705F7263746C5F726775693A2025750AEF
:100970002E737761705F6C616C745F6C6775693A38
:100980002025750A2E737761705F72616C745F72D7
:100990006775693A2025750A2E6E6F5F6775693A2B
:1009A0002025750A2E737761705F67726176655FC7
:1009B0006573633A2025750A2E737761705F6261F3
:1009C000636B736C6173685F6261636B73706163A7
:1009D000653A2025750A2E6E6B726F3A2025750ACE
:1009E0000064656275675F636F6E6669672E72612A
:1009F000773A20253032580A2E656E61626C653A6E
:100A00002025750A2E6D61747269783A2025750A61
:100A10002E6B6579626F6172643A2025750A2E6DBE
:100A20006F7573653A2025750A006565636F6E669C
:100A300069673A0A64656661756C745F6C617965B3
:100A4000723A2025750A003F000A6D6F7573653A8A
:100A5000206F66660A000A6D6F7573653A206F6EC7
:100A60000A000A6B6579626F6172643A206F66668C
:100A70000A000A6B6579626F6172643A206F6E0AD0
:100A8000000A6D61747269783A206F66660A000A1E
:100A90006D61747269783A206F6E0A000A6465624B
:100AA00075673A206F66660A000A64656275673A80
:100AB000206F6E0A000A0A4A756D70696E672074AD
:100AC0006F20626F6F746C6F616465722E2E2E20C2
:100AD00000433E2000436C656172696E67204545A6
:100AE00050524F4D0A000A002530325820006B65E5
:100AF00079626F6172645F7265706F72743A200020
:100B00005B735D005B575D005B535D005B525D0096
:100B10005B445D005B435D000C0341004D004A00F7
:100B2000360036000000180341004D004A004B001B
:100B30006500790062006F006100720064000000CF
:100B40000403090409025B00030100A0FA09040080
:100B500000010301010009211101000122400007E9
:100B600005810308000109040100010300000009D8
:100B70002111010001227B000705820320000109E9
:100B800004020002030000000921110100012222D9
:100B9000000705830320000107050303200001125D
:100BA00001000200000008EDFE66BD010001020028
:100BB000010631FF0974A1010975150026FF009592
:100BC00020750881020976150026FF00952075081A
:100BD0009102C005010902A10185020901A10005D8
:100BE00009190129081500250195087501810205DB
:100BF00001093009311581257F95027508810609A3
:100C0000381581257F950175088106050C0A380283
:100C10001581257F950175088106C0C005010980F1
:100C2000A101850319012AB700150126B700950116
:100C300075108100C0050C0901A101850419012A64
:100C4000A002150126A002950175108100C00501C2
:100C50000906A101050719E029E7150025019508F6
:100C6000750181029501750881010507190029FFA9
:100C7000150026FF00950675088100050819012951
:100C800005950575019102950175039101C0112427
:100C90001FBECFEFDAE0DEBFCDBF04B603FE18C043
:100CA0008091F9029091FA02A091FB02B091FC02AE
:100CB0008730904BA740B04B59F41092F902109234
:100CC000FA021092FB021092FC02E0E0F8E30995B0
:100CD00011E0A0E0B1E0EEE3FEE502C005900D9268
:100CE000AE3FB107D9F722E0AEEFB1E001C01D92EF
:100CF000A93FB207E1F70E948B180C941D2F0C94AA
:100D00000000FF93EF93E091FE01F091FF01309717
:100D100009F00995EF91FF910895FC0185918030CC
:100D200011F0EFDFFBCF0895FF27E0E230E247FF4D
:100D30000CC0419597FF09C0EDE2609570958095D4
:100D40009095611D711D811D911D27FF02C0219588
:100D500030E350E2AA27660F771F881F991FAA1F4A
:100D6000A41710F0A41B63955A95A9F7AA3008F0B0
:100D7000A95FA05DAF93F39561157105810591059C
:100D800041F7ED3211F4EF93F395F21718F43F9316
:100D9000F395FBCF8F91B5DFFA95E1F70895E991CF
:100DA000F9918591803021F0853219F0AADFF9CFD1
:100DB000089520E0E89455915532C1F3503311F471
:100DC000689455915A3348F4505390F3220F022EF1
:100DD000220F220F200D250FF4CF0EF421958991BB
:100DE0009991533619F3533729F1533559F1BC0111
:100DF00088279927E8945C3621F489919991689421
:100E00005591543639F446EF7EF077FF0DC08FEFE1
:100E10009FEF0AC055374AE039F0583540E121F0DC
:100E2000523642E009F00895FF93EF937DDFEF9192
:100E3000FF91B7CFFF93EF93FC0181918030B9F31D
:100E400060DFFBCFFF93EF9368DFF1CFDF93CF93AA
:100E5000CDB7DEB72596A3DFCF91DF91089581E06E
:100E6000089581E008950C94310708950C94350796
:100E70001F93CF93DF9300D000D01F92CDB7DEB782
:100E800049835A836B833091010289819A813111A0
:100E900014C0662359F0222349F00E94600E182FD7
:100EA000682F89819A810E94090E03C00E94340E26
:100EB000182F69817A81812F04C00E94600E698198
:100EC0007A810F900F900F900F900F90DF91CF913C
:100ED0001F910C94B015FC01262F40815181628135
:100EE000738184810C94380781E00895CF93DF9358
:100EF000EC0160E00E946B07BE01DF91CF910C9482
:100F000036070C943C170C94381708950E94B30CC4
:100F10000E9485072FEF84E39CE0215080409040A1
:100F2000E1F700C000000C949B260F931F93CF9312
:100F3000DF938C0161E00E946B07EC01B8010E9415
:100F40003307882309F462C0B801CE010E94571DFF
:100F5000882309F45BC0B801CE010E947A2488235B
:100F600009F454C0B801CE010E94401F882309F43F
:100F70004DC0B801CE010E94D623882309F446C093
:100F8000F80182818823D9F1CF3D8CE5D80779F12A
:100F900040F4C115FCE5DF0791F0C130DC4591F06C
:100FA0002EC0CC35EDE5DE0741F1CD35FDE5DF079F
:100FB00009F1CB35DD4519F50E94F71220C00E94DA
:100FC000860724C080919A02C82FC095C170C0FBCB
:100FD00080F980939A02CC2329F088E392E00E9462
:100FE0008D0614C086E292E00E948D0610C00E9419
:100FF000AB130CC00E94EE1202C00E94FA12C8018C
:10100000DF91CF911F910F910C942F07C0E08C2F8F
:10101000DF91CF911F910F9108950E94CF2580E01D
:101020000E94351E0C9450080E940F1C0E94530809
:101030000C94D5258295982F937344E0949F90014A
:1010400011248C7C86958695282B822F8575880F98
:101050002A7A2695822B0895CF93DF93D92F0E9469
:101060001A08C82F8D2F0E941A082C2F30E0322F1B
:101070002227A901482BCA01DF91CF910895089535
:101080000C943F0881E008950C9442080895CF9392
:10109000C82F0E9440088C2F0E944408CF910895C9
:1010A00080E00C9447080E94D6240C944708CF9304
:1010B0000E94D624C82F80910002C81741F1C09326
:1010C000000280919A0282FF1EC080FF04C080E56A
:1010D00092E00E948D0680919A0280FF0CC01F92C0
:1010E000CF938BE492E09F938F930E9426070F90FB
:1010F0000F900F900F9080919A0280FF04C089E4B6
:1011000092E00E948D068C2FCF910C944708CF91CE
:101110000895CF93DF93CDB7DEB72B970FB6F89432
:10112000DEBF0FBECDBF4F83588769877A878B8715
:1011300061110E9426129E012F5F3F4F86E0F90148
:1011400011928A95E9F785E0FE013796D901019061
:101150000D928A95E1F789819A814C815D81452BB9
:1011600031F09F3F31F491E08F3F19F403C091E0DB
:1011700001C090E090FF09C049815A816B817C8158
:101180008D819E810E94471105C0C9010E9474078C
:101190008111F2CF2B960FB6F894DEBF0FBECDBFF4
:1011A000DF91CF910895FC01808191810E94A20E70
:1011B0000895CF93882309F4A9C0C82F8238C1F4B9
:1011C0000E94D62481FDA2C069E380910201909122
:1011D00003010E94A7250E9448122FEF81EE94E0A0
:1011E000215080409040E1F700C0000069E319C041
:1011F000833801F50E94D62480FD88C063E5809184
:101200000201909103010E94A7250E9448122FEF2E
:1012100081EE94E0215080409040E1F700C0000052
:1012200063E580910201909103010E94A925CF916D
:101230000C9448128438C1F40E94D62482FD66C002
:1012400067E480910201909103010E94A7250E940A
:1012500048122FEF81EE94E0215080409040E1F75A
:1012600000C0000067E4DDCF8CEF8C0F813AF8F40A
:101270008C2F0E947F23811149C06C2F8091020125
:10128000909103010E947125882349F06C2F809171
:101290000201909103010E94A9250E9448126C2F1F
:1012A00080910201909103010E94A725C0CF80E2A6
:1012B0008C0F883048F4C77081E001C0880FCA9550
:1012C000EAF70E940912B3CFEBE5EC0FE33040F4EC
:1012D000F0E0E75BFE4F808190E0CF910C943925E0
:1012E000E8E5EC0FE73150F4F0E0EE0FFF1FE55EAC
:1012F000FE4F80819181CF910C944F25CD3E30F0EF
:101300008C2F0E941019CF910C94E219CF9108955F
:10131000882309F464C0823879F40E94D62481FFBE
:101320005EC069E380910201909103010E94A725AC
:101330000E94481269E310C08338B1F40E94D62499
:1013400080FF4DC063E580910201909103010E94EE
:10135000A7250E94481263E5809102019091030144
:101360000E94A9250C944812843879F40E94D6244E
:1013700082FF35C067E480910201909103010E94D1
:10138000A7250E94481267E4E7CF9CEF980F913A97
:1013900010F4682FE1CF90E2980F983050F48770E6
:1013A00091E001C0990F8A95EAF7892F0E940F12E8
:1013B000D9CF9BE5980F933020F480E090E00C9417
:1013C000392598E5980F973120F480E090E00C944F
:1013D0004F258D3E20F00E946B190C94E219089560
:1013E0001F93CF93DF93182FEB010E94D90820970A
:1013F00041F08FE99FE00197F1F700C000002197CD
:10140000F6CF812FDF91CF911F910C9488098933FA
:1014100019F060E070E002C060E570E00C94F00943
:10142000882321F00E9409120C9448120895882301
:1014300021F00E940F120C9448120895CF92DF926F
:10144000EF92FF920F931F93CF93DF937C01D62FE0
:10145000C72FFC011281058102950F700E94FF11B8
:101460008823B9F01123A9F08C2F807F803421F0DC
:1014700080E28D0F883068F08091D20282FD09C031
:1014800082E00E94A8120E94FF1191E0D82ED92676
:1014900001C0D12CCC2EC2948FE0C8228C2D90E0BC
:1014A0008C30910508F0CFC1FC01EA5AFF4F0C9433
:1014B000AE2E8C2F807FCF70882311F0C295C07F15
:1014C000112399F0CC2309F4AAC180E28D0F883052
:1014D00010F0D11104C08C2F0E94091203C08C2F70
:1014E0000E9419120E9448129AC18D2F0E948809E9
:1014F000CC2309F4A8C180E28D0F883038F1DD23B8
:1015000029F18C2F0E941F1224C08C2F807FCF7056
:10151000803211F0C295C07FDD2319F0D130A1F1E6
:101520003DC08091D20282FF17C0112349F0CC2325
:1015300029F08C2F0E9409120E94481280E070C18D
:1015400080E00E948809CC2309F47DC18C2F0E9481
:101550000F120E94481277C1112371F0002341F04D
:10156000013031F40E9429128C2B0E9431126BC180
:101570000E9429128C2B1DC0002319F0013009F4A0
:1015800062C10E943E1225C0112321F0063008F0EE
:101590005AC10EC0053008F056C11BC0112361F0BE
:1015A000002331F0F701858180FF39C18F70858379
:1015B0008C2F0E94100A47C1002359F0D93309F03B
:1015C0003FC1FFEF07EE13E0F15000401040E1F79C
:1015D00035C18C2F0E94170A36C18C2F86958695AF
:1015E000837019F0813061F02EC1112321F08D2F0D
:1015F0009C2F937002C080E090E00E9439252BC19F
:10160000112321F08D2F9C2F937002C080E090E079
:101610000E944F2520C18D2F112319F00E9410190F
:1016200002C00E946B190E94E21915C18C2F8370B1
:1016300009F047C011110BC12D2F22952695277057
:10164000220F220F6D2F6F70862F90E0A0E0B0E088
:10165000022E04C0880F991FAA1FBB1F0A94D2F73D
:10166000D4FF10C04FE050E060E070E004C0440FD1
:10167000551F661F771F2A95D2F7409550956095A4
:10168000709503C040E050E0BA01C695C695C3709E
:101690008A019B01082B192B2A2B3B2BC901B8016E
:1016A000C23049F058F4C13019F00E941F0DCFC06C
:1016B0000E940D0DCCC00E94310DC9C00E940B0DBF
:1016C000C6C0112319F08C2F817001C08695882324
:1016D00009F4BDC02D2F229526952770220F220FC9
:1016E0006D2F6F70862F90E0A0E0B0E0022E04C056
:1016F000880F991FAA1FBB1F0A94D2F7D4FF10C0EE
:101700004FE050E060E070E004C0440F551F661FDA
:10171000771F2A95D2F7409550956095709503C034
:1017200040E050E0BA01C695C695C3708A019B019E
:10173000082B192B2A2B3B2BC901B801C23049F0C9
:1017400058F4C13019F00E94E40D81C00E94D20DFE
:101750007EC00E94F60D7BC00E94450D78C0CF7000
:10176000112339F08C2F0E946B0D8D2F0E94100ACF
:101770006EC08D2F0E94170A8C2F0E948C0D67C09F
:10178000D23F21F128F4D03F41F0D13FC1F043C016
:10179000D33F19F1D43F79F03EC0112341F0053019
:1017A00008F051C08C2F8F710E94B10D4CC00630D3
:1017B00008F049C0F7CF8091D20282FF18C01123F0
:1017C00039F08C2F8F710E946B0D3DC01123C9F32E
:1017D0008C2F8F710E948C0D36C0112329F08C2F15
:1017E0008F710E94560D2FC00E94510D2CC01123E5
:1017F00049F0CF718C2F0E946B0D63E08C2F0E94FB
:101800008D1221C081E00E94A8120230E0F082E037
:101810000E94A81218C0112331F0002391F28D2FDD
:101820000E94D90810C0002399F2D93349F41FEF60
:1018300027EE33E0115020403040E1F700C00000B7
:101840008D2F0E94880988EF8C0D843020F40E942F
:10185000D6240E944708DD20C9F00E94FB1180FDBC
:1018600015C0F70112820E94F5110E946B0DC7018D
:101870000E94670C0E94F511DF91CF911F910F918B
:10188000FF90EF90DF90CF900C948C0DDF91CF9173
:101890001F910F91FF90EF90DF90CF9008950F93DD
:1018A0001F93CF93DF93EC01688179818A810E9435
:1018B000AD0E8C010E94080E0E94F90CB801CE01F9
:1018C0000E941E0ADF91CF911F910F910895CF932F
:1018D000DF93EC01988189812B813C81232B31F0AE
:1018E0008F3F31F481E09F3F19F403C081E001C0D4
:1018F00080E080FD1DC0CE010E949507811110C0BF
:101900000E94FF118823A1F08A81882389F08091A9
:10191000D20282FD0DC082E0DF91CF910C94A8121B
:10192000CE010E944F0CCE01DF91CF910C9476072F
:10193000DF91CF91089580E090E00E94392580E00A
:1019400090E00E944F250E9426120E9448120E9499
:10195000951B0C94E21980910201909103010E9461
:10196000AB250C949B0C0E9416120C94AB0C929518
:101970009F70963079F010F4925001C09A509230D6
:1019800068F4803F69F018F4883E40F409C0843F51
:1019900029F406C0883E20F0813F11F080E00895D0
:1019A00081E00895FC01808191810E94A20E0E9435
:1019B000B70C0895CF93DF9300D000D01F92CDB71E
:1019C000DEB70F900F900F900F900F90DF91CF9197
:1019D0000895CF93DF9300D000D000D0CDB7DEB70D
:1019E00026960FB6F894DEBF0FBECDBFDF91CF9124
:1019F0000895089508950C94FA0C0C94FB0C0E9421
:101A0000FD0C609338027093390280933A029093F0
:101A10003B020C949B0C0C94FF0C0F931F930091B2
:101A200038021091390220913A0230913B02602B2A
:101A3000712B822B932B1F910F910C94FF0C0F9302
:101A40001F93009138021091390220913A0230918F
:101A50003B0260237123822393231F910F910C94E7
:101A6000FF0C0F931F9300913802109139022091BF
:101A70003A0230913B0260277127822793271F91FA
:101A80000F910C94FF0C0C94FA0C0E94430D609380
:101A900034027093350280933602909337020C948F
:101AA0009B0C60E070E0CB010C94450D0F931F93ED
:101AB00041E050E060E070E08A019B0104C0000F4B
:101AC000111F221F331F8A95D2F7C901B8011F9138
:101AD0000F910C94450D0F931F9341E050E060E08F
:101AE00070E004C0440F551F661F771F8A95D2F718
:101AF0008091340290913502A0913602B091370264
:101B00008A019B01082B192B2A2B3B2BC901B801F9
:101B10001F910F910C94450D0F931F9341E050E0DE
:101B200060E070E004C0440F551F661F771F8A9560
:101B3000D2F74095509560957095809134029091C0
:101B40003502A0913602B09137028A019B01082329
:101B500019232A233B23C901B8011F910F910C942B
:101B6000450D0F931F9341E050E060E070E004C02A
:101B7000440F551F661F771F8A95D2F78091340254
:101B800090913502A0913602B09137028A019B01F3
:101B9000082719272A273B27C901B8011F910F9150
:101BA0000C94450D0F931F93009134021091350250
:101BB0002091360230913702602B712B822B932BB0
:101BC0001F910F910C94450D0F931F9300913402B8
:101BD0001091350220913602309137026023712333
:101BE000822393231F910F910C94450D0F931F9304
:101BF0000091340210913502209136023091370263
:101C000060277127822793271F910F910C94450D10
:101C1000089520E1929F800D1124E82FE695E69526
:101C2000E695877051E001C0550F8A95EAF785E087
:101C3000E89FF0011124EE5FFD4F20E030E070E0FE
:101C40004081CB01022E02C0969587950A94E2F757
:101C50008170819584278523842781932F5F3F4F4F
:101C60002530310569F7089520E1929F800D1124F8
:101C7000682F669566956695982F977085E0689FA2
:101C8000B001112440E050E080E0FB01E40FF51FBB
:101C9000EE5FFD4F208130E0092E02C0369527957A
:101CA0000A94E2F721703327042E01C0220F0A9410
:101CB000EAF7822B4F5F5F4F4530510531F70895AA
:101CC000BF92CF92DF92EF92FF920F931F93CF9329
:101CD000DF938C01C0903402D0903502E090360240
:101CE000F09037028091380290913902A0913A0227
:101CF000B0913B02C82AD92AEA2AFB2ACFE1D0E0D8
:101D0000D701C6010C2E04C0B695A7959795879567
:101D10000A94D2F780FD04C0219790F7B12C07C038
:101D2000BC2EB8018C2F0E94C5150197A9F38B2DED
:101D3000DF91CF911F910F91FF90EF90DF90CF90A7
:101D4000BF900895CF93DF93EC010E94600EBE0117
:101D50000E94C515DF91CF9108951F93CF93DF9314
:101D6000EB0190910102992321F0CB010E94A20E78
:101D700013C0882349F0CB010E94600E182F682FF2
:101D8000CE010E94090E04C0CB010E94340E182F10
:101D9000BE01812F0E94C515DF91CF911F9108953B
:101DA0001F93CF93DF93C0913C0216E080913D02D8
:101DB000C81799F0D0E01C9FF0011D9FF00D112471
:101DC000E25CFD4F40815181628173818481958104
:101DD0000E94E90C2196C770E9CFDF91CF911F9146
:101DE000089540916E0250916F026091700270915F
:101DF000710280917202909173020C94E90CEF923F
:101E0000FF920F931F93CF93DF938091730282957C
:101E10008F7009F065C080917002882309F460C05A
:101E200080913C02F0903D0210916E0200916F0291
:101E3000609171027091720291E01F3F09F090E091
:101E4000C0910001D0910101292F96E0E92E8F1554
:101E500009F446C06115710521F00F3F21F030E013
:101E600003C031E001C0322F90E030FD36C0E89E63
:101E7000F001E99EF00D1124DF01A25CBD4F119627
:101E80003C911197301329C03C91311326C0129612
:101E90003C911297311121C013964D915C9114978A
:101EA000461B570B4C175D07C0F4809173028F706F
:101EB000806180937302ED5BFD4F80818F70806144
:101EC00080838EE692E00E94670CDF91CF911F9194
:101ED0000F91FF90EF900C94D00E01968770B7CFC2
:101EE000DF91CF911F910F91FF90EF9008959F92F6
:101EF000AF92BF92CF92DF92EF92FF920F931F9318
:101F0000CF93DF93CDB7DEB761970FB6F894DEBFFE
:101F10000FBECDBF8C0185E0F801DE011D9601905A
:101F20000D928A95E1F7D8011296EC9090916E028D
:101F3000E0916F02209171023091720221153105FA
:101F400031F0EF3F31F481E09F3F19F403C081E0AD
:101F500001C080E0B82FB1709B2E80FD47C1D80131
:101F60004C9111965C9111971396AD90BC9014977B
:101F70008EE6C82E82E0D82EF0907002B501621B6A
:101F8000730B2091000130910101FF2009F4D9C0A9
:101F9000809173026217730708F095C0282F207F85
:101FA00009F052C05E1313C0491311C0FE2CE1109A
:101FB0000EC08F708061809373020E94F10EC60183
:101FC0000E94670C80917302F80185834DC1AB2894
:101FD00031F05F3F31F481E04F3F19F403C081E0FD
:101FE00001C080E080FD03C081E08E2502C080E05A
:101FF00090E0F82FF170FF2E80FF1CC080913C0212
:1020000020913D0236E0821709F40BC190E0389F21
:10201000F001399FF00D1124E25CFD4F61815613F0
:1020200006C06081461303C06281E61203C00196B8
:102030008770E9CFFE2CEE2009F416C1809173025F
:1020400081608093730254C05E1306C0491304C0BC
:10205000E11002C0F80199C0C8010E94D20C882387
:1020600061F1EE2051F120917302822F82958F70E1
:1020700090E0029774F080916E0290916F029887C1
:102080008F831986BB86AA862C87CE0107960E946D
:10209000670C86E0F801AEE6B2E001900D928A95F9
:1020A000E1F70E94FF0E0E94F10E0AC05E1711F1C7
:1020B000C8010E94D20C81112CC0C8010E94670C7B
:1020C000FF24F394D1C0282F207F81F77A2DB98A7D
:1020D000A88A6E2D89890E94DA0C8EE692E00E9411
:1020E000670C86E0D6011D928A95E9F70E94F10EF1
:1020F000F12CBAC04913DCCFE110DACFF8018583A7
:10210000C8010E94670C86E0D6011D928A95E9F706
:10211000ABC0EE2091F220917302822F82958F70D6
:1021200090E002970CF4B5CF80916E0290916F020F
:102130009A8389831B82BD82AC822E83CE01019655
:10214000A6CF6217730708F044C0FE2CEE2009F4F6
:10215000B4CF5E1330C049132EC02091730220FD0E
:1021600021C0822F82958F70482F50E04115510574
:10217000C9F0F80125834F30510541F08F5F982F4A
:102180009295907F822F8F70892B8583C8010E9442
:10219000670C86E0F801AEE6B2E001900D928A95F8
:1021A000E1F73CC086E0F801AEE6B2E001900D92A6
:1021B0008A95E1F759C0C8010E94D20C811169CFFC
:1021C00080917302816080937302C8010E94670C42
:1021D0004BC07A2DB98AA88A6E2D89890E94DA0CA3
:1021E00086E0D6011D928A95E9F718C0EE2009F421
:1021F00064CFC8010E94D20CF82E882309F45DCF69
:1022000086E0F801AEE6B2E001900D928A95E1F722
:102210008EE692E00E94D3080E94FF0E0E94F10E0B
:1022200023C04D875E878D859E850E94A20E292F33
:1022300022952F70223028F49F7039F0811105C04B
:102240000BC0243028F49F7049F4805E883020F061
:10225000C8010E94670C9F2CF92C06C0D801159666
:102260009C91907F91F7F8CF8F2D61960FB6F894DF
:10227000DEBF0FBECDBFDF91CF911F910F91FF90B9
:10228000EF90DF90CF90BF90AF909F9008951F93F5
:10229000CF93DF93CDB7DEB72C970FB6F894DEBFA0
:1022A0000FBECDBF4F83588769877A878B879C87FE
:1022B000CE0107960E94770F8823D1F09F818885F1
:1022C0002A853B85232B31F08F3F31F481E09F3FFE
:1022D00019F403C081E001C080E080FD47C04F8158
:1022E000588569857A858B859C850E94E90C3EC05E
:1022F00086E0FE013796DE01119601900D928A95D7
:10230000E1F7FF81E8856A857B856115710531F00C
:10231000EF3F31F481E0FF3F19F403C081E001C0D9
:1023200080E080FD23C020913D0230E0C90101968C
:102330008770992740913C0250E084179507F1F18E
:10234000F983EA837D836C8396E0929FD001939F0B
:10235000B00D1124A25CBD4FFE01319601900D928B
:102360009A95E1F780933D020E94D00E16E080918D
:102370003C0290913D02891771F1189FC001112410
:10238000825C9D4F0E94770F882329F1E0913C02E7
:102390001E9FF0011124E25CFD4F4081518162815A
:1023A0007381848195810E94E90C80913C0290E0C8
:1023B00001968770992780933C02D9CF0E94B30C75
:1023C00010923D0210923C02EEE6F2E086E0DF0160
:1023D0001D928A95E9F72C960FB6F894DEBF0FBED2
:1023E000CDBFDF91CF911F91089580917C0285959B
:1023F00085958595089580917C02877008959091C8
:102400007C02977081E009F480E008958091870252
:10241000089590918702892B809387020895809573
:1024200090918702892380938702089510928702F2
:10243000089590918602892B809386020895809555
:1024400090918602892380938602089510928602D5
:10245000089580917D02089508950C942C120C9497
:102460002D129091D20292FD08C090917D02981792
:1024700021F080937D020C942F12089580917D02AB
:10248000882329F010927D0280E00C942F12089589
:10249000CF93DF93E0910201F091030180918702D5
:1024A0008083E0910201F091030190818091860286
:1024B000892B808380917D02882381F0E091020145
:1024C000F09103019081892B80838091020190918A
:1024D00003010E94652581110E943E12C0910201F4
:1024E000D091030148E050E064E772E0CE010E9421
:1024F000CE2E892B69F088E0FE01A4E7B2E00190BE
:102500000D928A95E1F7CE01DF91CF910C94E224F0
:10251000DF91CF9108950C942C129091D20292FDEC
:1025200010C098E0899F90011124262B20937C02F3
:102530000E946B0D80917C028595859585950C9404
:102540008B120C946B0D10927C0280E00C948B1219
:1025500020917C028095822380937C02982F977033
:1025600099F430E0482F082E000C550B241735073E
:1025700059F09091D20292FD07C085958595859579
:102580000E948C0D0C94A3120895CF939091D202C7
:1025900092FB222720F92817F9F0C82F892FC0FBBA
:1025A00082F98093D2028091D1029091D2020E944E
:1025B000271382E00E94A81280919A0280FF0CC02B
:1025C0001F92CF938BE592E09F938F930E942607F3
:1025D0000F900F900F900F90CF9108958091D2029D
:1025E00082FB882780F991E089270C94C51281E04D
:1025F0000C94C51280E00C94C5126FEF7FEF80E061
:1026000090E00C94072F80E090E00E94E32E21E000
:10261000893E9E4F09F020E0822F089582E090E0ED
:102620000C94DB2E83E090E00C94DB2ECF9384E0BF
:1026300090E00E94DB2EC82F82E290E00E94DB2E09
:102640002C2F30E0A901582BCA01CF910895CF93C8
:10265000C92F682F84E090E00E94E92E6C2F82E25F
:1026600090E0CF910C94E92EAB01BC018FE090E09B
:102670000C94FB2EAB01BC0183E190E00C94FB2E8B
:1026800060E070E0CB010C943A1360E070E0CB01A5
:102690000E9434130C94401369EE7EEF80E090E0CA
:1026A0000E94072F60E082E090E00E94E92E60E047
:1026B00083E090E00E94E92E1092380210923902D5
:1026C00010923A0210923B0260E084E090E00E9497
:1026D000E92E60E082E290E00E94E92E60E085E071
:1026E00090E00E94E92E60E086E090E00E94E92EF2
:1026F0006FEF87E090E00E94E92E40E050E0BA01E1
:1027000088E090E00E94FB2E60E08DE090E00E9467
:10271000E92E40E050E0BA0188E190E00E94FB2EF3
:1027200060E087E190E00E94E92E40E050E0BA01CD
:102730008CE190E00E94FB2E60E070E080E290E08F
:102740000E94072F40E050E0BA0188E190E00E942B
:10275000FB2E0C9445130C944C13682F8EE090E0E4
:102760000C94E92E0E945A26609396027093970269
:1027700080939802909399026093920270939302CF
:102780008093940290939502089585B7806885BFE1
:1027900085B7806885BF089581E008950C94CC13B7
:1027A00008950C94D0130C94D0130C94D3130C9460
:1027B000D0130C94D7130C94D0130E94C51382E944
:1027C00098E20E94CC240E94DB130C94D9130E943F
:1027D000D1130C94D0130E94B9160E9446080C9491
:1027E0002A1F0E9445260E94E4170E94EB130E94B4
:1027F0000F1C0C94D5135F926F927F928F929F92D1
:10280000AF92BF92CF92DF92EF92FF920F931F93FE
:10281000CF93DF93CDB7DEB72A970FB6F894DEBF1C
:102820000FBECDBF0E94F917C82E81110E94B213AE
:1028300038E8832E32E0932E00E010E0502E802FF7
:102840000E94DD165C01F401619071904F016826D1
:10285000792661147104B1F40F5F1F4F0530110523
:1028600069F78FEF89838A831B820E944E268160DD
:10287000782F9D838C8349815A816B818D810E9441
:1028800089083AC080919A0281FD0E94E616D12CF7
:10289000EE24E394F12CC3018E219F21892B29F191
:1028A0000E94CE138823A9F0DE825F82AE20BF2073
:1028B00081E0AB2809F480E088870E944E26816081
:1028C000782F9A8789874E815F8168858A850E94E3
:1028D0008908000F111FF801E857FD4F8081918191
:1028E000E826F926F182E08207C0D394EE0CFF1CA3
:1028F000F0E1DF12D0CFB0CF81E0C11001C080E0A5
:102900002A960FB6F894DEBF0FBECDBFDF91CF91F0
:102910001F910F91FF90EF90DF90CF90BF90AF90FD
:102920009F908F907F906F905F9008950E94FB130F
:102930000E947D1E0E94821A0C945708CF93DF9349
:102940000E94CA15EC01811521E5920708F045C0E7
:10295000811530E5930708F094C0883E910528F56D
:10296000803E910508F0F8C0883A910570F4853AE8
:10297000910508F07CC08130910509F475C008F418
:10298000E8C0049708F0E8C0E4C08F3B910508F068
:10299000E0C0C85AD0E0CC0FDD1FC45BDE4F099009
:1029A000D881C02DCE019464D8C0811540E294072F
:1029B00058F4811551E0950708F0CEC08D3E910581
:1029C00008F4C7C09065C9C0C11580E4D80708F4F1
:1029D000C0C0DF70CE01906AC0C0811525E59207A6
:1029E000A8F4811534E5930708F095C0811543E5F7
:1029F000940708F07BC0811552E5950708F061C087
:102A0000D82FCC27CE01816F906AA7C0C11589E568
:102A1000D807A0F4C11528E5D20708F082C0C11577
:102A200036E5D30708F095C08C2F0E945E168F7193
:102A300090E0D82FCC27CE0190628FC0C1154AE517
:102A4000D40708F474C0CE0190568115904208F066
:102A500080C08D2F8F710E945E16DD27D0628F712E
:102A6000AE01582BCA0179C081E090E076C0C55A0A
:102A7000D0E0C658DE4F8881C82FD0E0CE019064E8
:102A80006CC074E0969587957A95E1F7282F2370AE
:102A90003C2F337081E090E002C0880F991F3A9577
:102AA000E2F79C68AC01522B9A019C2F9F7096957F
:102AB000969550E2959FE0011124C9018C2B9D2B26
:102AC0004CC08370992721E030E002C0220F331FF1
:102AD0008A95E2F79C2F9695969580E2989FE00163
:102AE0001124C22BD32BCE019C6837C08370992749
:102AF00021E030E002C0220F331F8A95E2F79C2FBD
:102B00009695969540E2949FE0011124C22BD32B19
:102B1000CE019A6822C0D82FCC27CE01846F906A4C
:102B20001CC0DC2FCC27CE01806F906A16C08C2F82
:102B30008F700E945E1694E0D695C7959A95E1F73E
:102B4000CF70D0E0DC2FCC27D0699E01282BC901A3
:102B500004C080E090E001C0CE01DF91CF910895E4
:102B6000E72FF0E095E0899FE00DF11D112484E04E
:102B7000EE0FFF1F8A95E1F7E60FF11DEE0FFF1F25
:102B8000EA51FF4F8591949108950E94B0150E94DB
:102B90009E1408958238910569F1B0F4813391054E
:102BA00009F46DC048F48932910509F463C08A3292
:102BB000910509F469C008958533910509F455C05C
:102BC00089339105B9F00895833E910569F138F490
:102BD000803E9105B1F0823E910509F10895863E4F
:102BE0009105A9F1873E9105B9F1843E910509F05F
:102BF00064C023C02091D10220FD4FC021FD4DC0F3
:102C000008958091D10280FD44C08091D20280FF5E
:102C100044C08091D10284FD42C083EE4DC08091BA
:102C2000D10282FF38C0F5CF8091D10282FD33C03E
:102C30008091D20280FD31C0ECCF8091D20281FF21
:102C400032C08091D10284FD2AC087EE35C08091C8
:102C5000D10283FF26C0F5CF8091D10283FD21C030
:102C60008091D20281FD1FC0ECCF8091D10285FD01
:102C70001CC01DC08091D10285FD19C016C0809175
:102C8000D10286FD16C017C08091D10286FD13C007
:102C900010C089E311C082EE0FC080EE0DC080E04D
:102CA0000BC086EE09C084EE07C089E205C085E34B
:102CB00003C08AE201C081E390E008959091D102BF
:102CC00092FF0DC0282F2871283019F4877F846067
:102CD00006C0282F2471243011F48B7F886093FF65
:102CE0000DC0282F2871283119F4877E846106C011
:102CF000282F2471243111F48B7E88612091D20217
:102D000020FF0DC0382F3871383019F4877F81606B
:102D100006C0382F3171313011F48E7F886021FF69
:102D20000DC0282F2871283119F4877E816106C0D3
:102D3000282F2171213111F48E7E886194FD877EC8
:102D400008950C94FD120E94F9178FE39CE90197F6
:102D5000F1F700C000000E94F91780E00E94DD1624
:102D600080FF04C00E94A1160C949B2608950C9429
:102D7000A3160E940313811102C00E94AB130E948C
:102D80000E1380939A020E9416139093D20280939E
:102D9000D1020E94B7160E941213682F70E080E0E3
:102DA00090E00E940B0D6091340270913502809189
:102DB0003602909137020C94430DE82FF0E0EE0FAD
:102DC000FF1FE352FD4F808191810895CF92DF92E2
:102DD000EF92FF920F931F93CF93DF9380E892E0DF
:102DE0000E948D068DEDE82E82E0F82EC0E0D0E046
:102DF0009BE7C92E92E0D92E02E712E0DF93CF9332
:102E0000DF92CF920E94260788E792E00E948D060B
:102E1000F701819191917F010E942C089F938F93DC
:102E20001F930F930E94260780E792E00E948D0671
:102E300021968DB79EB708960FB6F8949EBF0FBE29
:102E40008DBFC530D105D1F6DF91CF911F910F9184
:102E5000FF90EF90DF90CF90089580EA8A95F1F788
:102E6000089500C008950C942D1708950C943517FB
:102E70000C9436170C9435170C943A17F894E82FE5
:102E8000E295EF70F0E031A1282F2F7081E090E003
:102E900001C0880F2A95EAF7982F9095932391A364
:102EA00092A1892B82A3789408950F931F93CF93B7
:102EB000DF93CDE8D1E089918F3F11F00E943E175A
:102EC00081E0C239D807B9F7CDE7D1E00DE811E0CC
:102ED00089918F3F11F00E943E170C171D07C1F713
:102EE000DF91CF911F910F910895BF92CF92DF9202
:102EF000EF92FF920F931F93CF93DF938C01C62F16
:102F0000D0E0CE0183579E4F6C01FC0190819F3F22
:102F100009F450C0B62EF894E92FE295EF70F0E076
:102F200081A19F7021E030E001C0220F9A95EAF75D
:102F3000822B81A382A12095282322A378940E942A
:102F40003117EDE7F1E04DE851E021E030E0E12C10
:102F5000F12C61916F3F89F0A62FA295AF70B0E080
:102F600090968C9190E06F7002C0959587956A95C8
:102F7000E2F780FD02C0C90102C080E090E0E82ACB
:102F8000F92A220F331F4E175F0719F7F6018081C8
:102F90008F3F11F00E943E1761E0E114F10409F443
:102FA00060E08B2D0E943317CC0FDD1FC00FD11FA7
:102FB000F982E882DF91CF911F910F91FF90EF90FE
:102FC000DF90CF90BF9008950E9455178AE0EDEDF5
:102FD000F2E0DF01982F1D929A95E9F7E3EDF2E018
:102FE000DF011D928A95E9F785E00E9444180C9450
:102FF0008107FF920F931F93CF93DF93CDB7DEB777
:103000002A970FB6F894DEBF0FBECDBF8E010F5FBB
:103010001F4F8AE0F80111928A95E9F7F12C6F2D84
:10302000C8010E947517F394F5E0FF12F8CF4AE04B
:1030300050E0B80183ED92E00E94CE2EFF24F3947D
:10304000009709F4F12C892B41F08AE0F801A3EDF7
:10305000B2E001900D928A95E1F72F2D45E06DEDDC
:1030600072E083ED92E00E9445180E9483078F2D45
:103070002A960FB6F894DEBF0FBECDBFDF91CF9179
:103080001F910F91FF9008950895FF920F931F9342
:10309000CF93DF93F82E092F162FD72FC42F22237B
:1030A00049F081E080939D020E944E2690939C02FD
:1030B00080939B0280919D028823D9F080919B028E
:1030C00090919C020E946626059798F0EF2DF02FB4
:1030D000A12FBD2F80E090E04C2F50E08417950782
:1030E00034F4219131912D933D930196F7CF1092B5
:1030F0009D02DF91CF911F910F91FF9008950E9443
:103100000E290E94F1130C941A290E941E290E9474
:1031100096140C943C290E94EC250E94F5280E94EC
:10312000DD130E947F180E9485180E94E713FBCFD1
:103130008091A40280FF06C06091090170E0660FD3
:10314000771F26C081FF04C06091090184E005C09B
:1031500082FF07C06091090188E0689FB0011124D7
:1031600017C09091A3029923D1F06091080196179E
:1031700088F72091090188E0289F90011124929FEF
:10318000A001939F500D112470E0CA010E94782E77
:103190006038710540F46115710519F406C068E0E6
:1031A00070E0862F08958FE7089581E0089580915B
:1031B000A40280FF08C06091050170E075956795D5
:1031C0007595679521C081FF06C06091050170E08B
:1031D0007595679519C082FF04C06091050170E084
:1031E00010C09091A202992399F060910401961762
:1031F000A0F780910501899FC001112470E00E9411
:10320000782E6038710540F46115710519F406C017
:1032100061E070E0862F08958FE7089581E00895BA
:103220008D3E21F40E949818819504C08E3E29F4A9
:103230000E9498188093A80208958F3E21F40E945E
:103240009818819504C0803F29F40E9498188093B3
:10325000A7020895893F19F40E94D71805C08A3F34
:1032600031F40E94D71881958093A90208958B3F6D
:1032700021F40E94D718819504C08C3F29F40E9444
:10328000D7188093AA0208959FE0980F983078F499
:1032900021E030E0A90102C0440F551F9A95E2F7E2
:1032A000CA019091A602892B8093A60208958D3FB2
:1032B00021F48091A40281600BC08E3F21F48091A3
:1032C000A402826005C08F3F29F48091A40284602B
:1032D0008093A40208958D3E39F49091A80297FF3F
:1032E00035C01092A80259C08E3E29F49091A802D0
:1032F0001916BCF32BC09091A7028F3E29F497FFBB
:1033000025C01092A70249C0803F19F41916CCF3CA
:103310001DC09091A902893F29F41916BCF410929E
:10332000A9023BC08A3F19F497FF10C0F8CF8B3F2A
:1033300039F49091AA0297FF09C01092AA022DC0F9
:103340008C3F21F49091AA021916BCF39FE0980FCC
:10335000983080F421E030E0A90102C0440F551FED
:103360009A95E2F7CA0180959091A60289238093ED
:10337000A60213C08D3F21F48091A4028E7F0BC062
:103380008E3F21F48091A4028D7F05C08F3F29F4E8
:103390008091A4028B7F8093A4028091A702811167
:1033A00006C08091A802811102C01092A3028091F0
:1033B000A902811106C08091AA02811102C0109257
:1033C000A202089580919A0283FF7EC08EEB92E064
:1033D0000E948D068091A6021F928F9389EB92E046
:1033E0009F938F930E94260787EB92E00E948D06A1
:1033F0008091A702282F082E000C330B3F938F9348
:1034000084EB92E09F938F930E94260782EB92E0D9
:103410000E948D068091A802282F082E000C330BE5
:103420003F938F938FEA92E09F938F930E9426079A
:103430008DEA92E00E948D068091A902282F082E25
:10344000000C330B3F938F938AEA92E09F938F9304
:103450000E94260788EA92E00E948D068091AA02C7
:10346000282F082E000C330B3F938F9385EA92E0B0
:103470009F938F930E94260782EA92E00E948D0616
:103480008091A3021F928F938FE992E09F938F9375
:103490000E9426078DE992E00E948D068091A40289
:1034A0001F928F938AE992E09F938F930E94260741
:1034B00087E992E00E948D068DB79EB74C960FB6B5
:1034C000F8949EBF0FBE8DBF0E944E262091A7028A
:1034D000211104C02091A802222321F09093A1027F
:1034E0008093A0022091A902211104C02091AA0278
:1034F000222321F090939F0280939E0285EA92E01E
:103500000C942B25EF92FF920F931F93CF93DF9391
:1035100000D000D000D0CDB7DEB786E0E5EAF2E01B
:10352000DE01119601900D928A95E1F7E090A702D5
:10353000F090A8020091A9021091AA021092A7028D
:103540001092A8021092A9021092AA02E11003C0E0
:10355000FF2009F45DC08091A0029091A1020E9419
:103560006626AC019091A302992339F020910A01BB
:1035700030E02417350758F04BC020910B018AE04A
:10358000289F900111242417350718F041C09F3F50
:1035900019F09F5F9093A302EE2061F00E949818AB
:1035A0001E1414F09FEF01C091E0989F902D1124FC
:1035B0009093A702FF2061F00E9498181F1414F046
:1035C0009FEF01C091E0989F902D11249093A80245
:1035D0003091A7023323E1F02091A8022223C1F009
:1035E00045EB3403C0011124992319F09093A702ED
:1035F00003C081E08093A70235EB2303C0011124AF
:10360000992319F09093A80203C081E08093A80247
:10361000011103C0112309F45DC080919E029091B5
:103620009F020E946626AC019091A202992339F074
:103630002091060130E02417350758F04BC0209147
:1036400007018AE0289F900111242417350718F0FC
:1036500041C09F3F19F09F5F9093A202002361F049
:103660000E94D718101614F09FEF01C091E0989FA8
:10367000902D11249093A902112361F00E94D71874
:10368000111614F09FEF01C091E0989F902D112426
:103690009093AA023091A9023323E1F02091AA026B
:1036A0002223C1F045EB3403C0011124992319F002
:1036B0009093A90203C081E08093A90235EB230314
:1036C000C0011124992319F09093AA0203C081E04C
:1036D0008093AA028091A70281110BC08091A80259
:1036E000811107C08091A902811103C08091AA02B3
:1036F00081110E94E219EB82FC820D831E8386E019
:10370000FE013196A5EAB2E001900D928A95E1F7AB
:1037100026960FB6F894DEBF0FBECDBFDF91CF91D6
:103720001F910F91FF90EF900895E5EAF2E086E097
:10373000DF011D928A95E9F71092A3021092A2026E
:103740001092A402089586E090E00C94DB2E682F7E
:1037500086E090E00C94E92E8091E7028470896104
:103760008093E7020C94A71B8091E70286958695CB
:10377000869508958091E70281FD13C08260809351
:10378000E7020E94A71B80919A0280FF08C08EEF7B
:1037900092E09F938F930E9426070F900F900C94B6
:1037A0007E1E08958091E70281FF13C08D7F809374
:1037B000E7020E94A71B80919A0280FF08C081EE59
:1037C00092E09F938F930E9426070F900F900C9486
:1037D000881E0895CF93C091E702C695C17080916D
:1037E0009A0280FF0CC01F92CF938AE193E09F93CF
:1037F0008F930E9426070F900F900F900F90CC236D
:1038000019F0CF910C94D21BCF910C94BA1B8091DC
:10381000E70286958170089580910C0108950E94B9
:103820000313811104C00E94AB130E94AC1B0E94C1
:10383000A31B8093E702282F26952695269530E036
:103840002430310524F0877088618093E7028091ED
:10385000E70280FF04C086958695869501C080E0CA
:103860000C94351E2091E702822F869586958695C9
:10387000482F50E04330510554F48F5F982F990F33
:10388000990F990F822F8770892B8093E70280917F
:10389000E70281608093E7020E94A71B80919A0251
:1038A00080FF11C08091E7028695869586951F92CC
:1038B0008F9381EA93E09F938F930E9426070F9046
:1038C0000F900F900F908091E702869586958695D0
:1038D0000C94351E8091E702982F969596959695B3
:1038E000A1F0915E990F990F990F8770892B8093A2
:1038F000E702887F91E009F490E08091E70290FB75
:1039000080F98093E7020E94A71B80919A0280FFB2
:1039100011C08091E7028695869586951F928F93B8
:1039200089E893E09F938F930E9426070F900F9052
:103930000F900F908091E7028695869586950C945E
:10394000351E8091E70280FD1FC081608093E702F1
:10395000813019F489E08093E7028091E7020E94A8
:10396000A71B80919A0280FF08C081E693E09F9395
:103970008F930E9426070F900F908091E702869503
:10398000869586950C94351E08958091E70280FFF8
:1039900014C08E7F8093E7020E94A71B80919A0239
:1039A00080FF08C08EE493E09F938F930E942607C8
:1039B0000F900F9080E00C94351E0895CF93C09126
:1039C000E702C17080919A0280FF0CC01F92CF93D2
:1039D00083E793E09F938F930E9426070F900F90A9
:1039E0000F900F90CC2319F0CF910C94C51CCF9160
:1039F0000C94A11C9091E702892F86958695869557
:103A00008F5F8F719770843038F4880F880F880F1C
:103A1000892B8093E70202C09093E7028091E7022E
:103A2000887F91E009F490E08091E70290FB80F9B3
:103A30008093E7020E94A71B80919A0280FF11C029
:103A40008091E7028695869586951F928F938AE3EB
:103A500093E09F938F930E9426070F900F900F90F3
:103A60000F908091E7028695869586950C94351E79
:103A7000843008F083E09091E7029770282F220F9E
:103A8000220F220F922B9093E702987F21E009F4F6
:103A900020E09091E70220FB90F99093E7020C94CC
:103AA000351E0E94381D8091E7020C94A71BFC0173
:103AB000DB0112968C918823F9F0EC5BFC45E73032
:103AC000F105D8F4EE59FF4F0C94AE2E83E001C0FF
:103AD00080E00E94511D80E008950E946A1CFBCF87
:103AE0000E94321CF8CF0E94DE1CF5CF0E94FA1C07
:103AF000F2CF0E94EA1BEFCF81E00895549A5C98C0
:103B000008955C9A08955C9808958F929F92AF9261
:103B1000BF92CF92DF92EF92FF920F931F93CF93BA
:103B2000DF938C0180918600909187006CE070E0BB
:103B30000E94642E6017710730F0C80169E070E0E0
:103B40000E94642E60C08091860090918700E09072
:103B50008600F0908700E0918600F0918700C6E033
:103B6000D0E0BE010E94642E20E030E0060F171F57
:103B7000211D311D4801590185E0880C991CAA1CA2
:103B8000BB1C8A95D1F7C701BE010E94642E6F014C
:103B9000E12CF12CA7019601260F371F411D511D65
:103BA000C501B4010E948C2E69017A01E091860062
:103BB000F0918700CA01B9010E94482E9B01AC0117
:103BC000DF010E94C32E9B01AC01C701B6010E9418
:103BD000482EDC01CB012FE0B695A79597958795E8
:103BE0002A95D1F7009186001091870020E030E0FF
:103BF000081719072A073B0728F46091860070917F
:103C00008700CB01BC01CB01DF91CF911F910F91B8
:103C1000FF90EF90DF90CF90BF90AF909F908F90EC
:103C200008951F920F920FB60F9211242F933F9376
:103C30004F935F936F937F938F939F93AF93BF93B4
:103C4000EF93FF930E94831DFF91EF91BF91AF917E
:103C50009F918F917F916F915F914F913F912F91A4
:103C60000F900FBE0F901F901895CF93C82F8430E0
:103C7000A8F4811114C08091880090918900892B4B
:103C800051F080916F008D7F80936F0080916F0065
:103C90008E7F80936F000E94831D11C0C3E08091CE
:103CA000880090918900892B51F480916F00826087
:103CB00080936F0080916F00816080936F00A0916E
:103CC0008600B09187002C2F30E00E94B42E23E0B4
:103CD00030E040E050E00E948C2EB42FA32F922FB2
:103CE0008827892F9A2FAB2FBB270E94851D909381
:103CF000890080938800CF91089508951092AD02B5
:103D00001092AC021092AE0281E08093AB02089553
:103D10001092AB020E94B41B0C94351E0F931F939C
:103D2000CF9380910D0191E0980F823019F090931C
:103D30000D0152C081E080930D010E940C1CC82F20
:103D40000091AC021091AD020F5F1F4F0E940C1C3E
:103D500028E7829FB0011124C8010E94642E90932D
:103D6000AD028093AC0228E7C29FB0011124660F18
:103D7000672F661F770B71950E94642E6F77809175
:103D8000AE02823019F4603439F404C0813021F479
:103D90006F3711F41092AB02E62FF0E0E754FC4FBE
:103DA000C49100918600109187000E94B41B282FB7
:103DB000C09FC001C19F900D11246DEF72E00E9461
:103DC000642E269FC001279F900D11240E94851DFF
:103DD0009093890080938800CF911F910F9108954F
:103DE0001F920F920FB60F9211242F933F934F9370
:103DF0005F936F937F938F939F93AF93BF93EF9353
:103E0000FF938091AB0281110E948E1E2091880049
:103E10003091890080918600909187006AEF70E070
:103E20000E94642E6B5F7F4F6217730710F40E942D
:103E3000811DFF91EF91BF91AF919F918F917F91E4
:103E40006F915F914F913F912F910F900FBE0F9007
:103E50001F9018950E947E1D82E08093800089E16A
:103E6000809381008FEF9FEF90938700809386006F
:103E70000E940F1C0E94071C81110C947E1E089545
:103E8000CF93DF93EC01FB018281882309F43CC1CD
:103E9000C430FDE5DF0760F4CB3F9CE5D90788F42B
:103EA0009E0122503C452431310508F02EC109C045
:103EB000C236EDE5DE0729F0C63AFDE5DF0709F079
:103EC00024C10E9416139093D2028093D102C13173
:103ED0008CE5D80709F4C6C008F042C0C930ECE54B
:103EE000DE0709F49BC000F5C5308CE5D80709F45E
:103EF00085C078F4C330ECE5DE0709F478C008F03B
:103F00007AC0C230DC4509F0F5C08091D1028160F1
:103F1000EFC0C7309CE5D90709F478C008F07AC033
:103F20008091D1028061E4C0CD30FCE5DF0709F467
:103F300087C058F4CB309CE5D90709F479C008F064
:103F40007BC08091D10288606FC0CF30FCE5DF0775
:103F500009F480C008F082C08091D102877FC8C078
:103F6000CE3F9CE5D90709F471C000F5C531FCE5E9
:103F7000DF0709F485C068F4C3319CE5D90709F46B
:103F800075C008F095C00E94B30C8091D1028F7764
:103F9000AFC0CC3FFCE5DF07A9F108F054C0CB3F30
:103FA000DC4509F0A7C08091D20240C0C230EDE5E7
:103FB000DE0709F489C058F4C1158DE5D80709F466
:103FC0005AC008F069C08091D20282602FC0C23608
:103FD000EDE5DE0709F47CC0C63AFDE5DF0709F42C
:103FE00081C0C330DD4509F085C080E06EC080919E
:103FF000D10282607DC08091D10216C08091D10231
:10400000886076C08091D20282604FC08091D102D8
:1040100080626EC08091D10280646AC00E94B30C3D
:104020008091D102806864C0846062C081603DC0BC
:104030008091D1028E7F5CC08091D1028D7F58C06B
:104040008091D10216C08091D20218C08091D20214
:104050008D7F2BC08091D1028F7E4AC08091D1028A
:104060008F7D46C08091D1028F7B42C08091D1026A
:10407000877F8B7F3DC08091D2028D7F8E7F15C060
:104080008091D10282FB222720F991E0922790FBB8
:1040900082F990FB83F92CC08091D202982F9095E1
:1040A00091708E7F892B90FB81F98093D20222C080
:1040B0000E94B30C8091D10287FB222720F991E066
:1040C000922790FB87F914C081E00E94AD1312C0C3
:1040D0008091D10284FB222720F991E0922790FB66
:1040E00084F906C08091D102982F909590FB80F9B9
:1040F0008093D1028091D1029091D2020E94271325
:104100000E94B30C80E001C081E0DF91CF9108955F
:10411000809104011F928F93809105011F928F93CC
:10412000809108011F928F93809109011F928F93B4
:1041300080910A011F928F9380910B011F928F93A0
:1041400089E394E09F938F930E9426078DB79EB7D3
:104150000E960FB6F8949EBF0FBE8DBF089588329D
:1041600020F58E3108F068C08B3091F1C0F48730B3
:1041700009F0BEC081E080930B0184E180930A01C5
:104180008AE0809309018EE18093080188E08093A2
:10419000050188E2809304018BE995E0C6C0833174
:1041A00009F443C0843169F1A3C08F3409F49EC07F
:1041B00028F4893231F1883359F09AC0813531F0D1
:1041C00008F4D4C0823509F4A7C092C08FEFA5C00F
:1041D0008DEB95E00E948D060E9488201F9281E061
:1041E0008F931F9288E08F9386EB94E09F938F9339
:1041F0000E9426070F900F900F900F900F900F9036
:1042000096C08AEB95E00E948D068091B3028823C8
:1042100009F4AAC01092B3021092B2021092B10235
:104220001092B0021092AF02B1C08CEA95E00E94E9
:104230008D060E9488207BC08D518093B30283300D
:1042400031F170F48130D1F0823009F03FC08AE062
:1042500091E09093B2028093B1028FE991E01FC088
:10426000853059F108F1863089F584E091E090932A
:10427000B2028093B1028AED91E011C08BE091E02F
:104280009093B2028093B10286E991E008C089E080
:1042900091E09093B2028093B1028BEA91E0909307
:1042A000B0028093AF0218C088E091E09093B20210
:1042B0008093B10288EB91E0F2CF85E091E090939A
:1042C000B2028093B10287EC91E0E9CF1092B30281
:1042D00089EA95E00E948D068091B302882309F453
:1042E00055C01F928F9385EA95E00DC08AE015C0F6
:1042F00088E995E01AC097FF47C0108280811F921D
:104300008F9382E995E09F938F930E9426070F90E9
:104310000F900F900F900BC081E0E091B102F091EF
:10432000B202309729F58FE895E00E948D06209122
:10433000B302222359F18091AF029091B00200970D
:1043400011F482E991E09F938F931F922F9386E857
:1043500095E09F938F930E9426070F900F900F90E8
:104360000F900F900F9016C080E0089586EFD5CF84
:104370002081082E000C990B820F911D8F3F910513
:1043800009F00CF4B8CF8FEF8083B8CF82E895E0C6
:104390000E948D0681E00895CF93C82F1F928F93BE
:1043A00083ED95E09F938F930E94260781E090E034
:1043B000A0E0B0E0BC01CD0104C0660F771F881FEC
:1043C000991FCA95D2F70E940B0D0F900F900F9076
:1043D0000F90CF910C94B30CEF92FF920F931F9319
:1043E000CF93DF938B3109F409C108F0AAC08B3059
:1043F00009F4CDC008F094C0863009F4CBC020F495
:10440000853009F4D9C06AC1873009F4DCC088302E
:1044100009F064C10E9412131F928F938AE29AE0FE
:104420009F938F930E9426070E940E1383FB992768
:1044300090F91F929F9382FB992790F91F929F9367
:1044400081FB992790F91F929F93982F91701F924B
:104450009F931F928F9381EE99E09F938F930E9479
:1044600026070E94161387FB222720F91F922F93FD
:1044700086FB222720F91F922F9385FB222720F904
:104480001F922F9384FB222720F91F922F9383FBE7
:10449000222720F91F922F9382FB222720F91F92B7
:1044A0002F9391FB222720F91F922F93292F217000
:1044B0001F922F9381FB222720F91F922F93282FE1
:1044C00021701F922F939F938F938CEF98E09F936F
:1044D0008F930E9426078DB79EB788960FB6F894E3
:1044E0009EBF0FBE8DBF0E94A31B982F96959695D9
:1044F00096951F929F93982F91701F929F931F9252
:104500008F9389EC98E09F938F930E9426078DB735
:104510009EB708960FB6F8949EBF0FBE8DBF35C0EC
:10452000803109F495C020F48E3009F47BC0D6C0E8
:10453000863109F4A8C0893109F0D0C083E496E03F
:1045400084C08A32E1F060F4873209F4C3C028F4F1
:104550008E3108F4C3C08D51BEC0893269F1BEC02E
:10456000833448F48A3308F0B3C0853309F4B2C009
:10457000883369F0B3C0833409F4ACC0AFC085EDB3
:104580009AE00E948D060E94AB13C1E0ACC086E2A7
:1045900097E05BC080919A02817F8E7F80939A0220
:1045A0008FEF96E00E948D0681ED9AE00E948D06C5
:1045B00081E08093B402E9CF85EB9AE00E948D06FA
:1045C0000E948607E2CF80919A02C82FC095C170E1
:1045D000C0FB80F980939A02CC2329F089EA9AE003
:1045E0000E948D0680C08CE99AE00E948D06809121
:1045F0009A02897F877F80939A02C7CF90919A020F
:1046000091FBCC27C0F981E0C827892FC0FB81F935
:1046100080939A02CC2319F08FE89AE029C081E8B0
:104620009AE013C090919A0292FBCC27C0F981E0E6
:10463000C827892FC0FB82F980939A02CC2319F0F6
:1046400082E79AE015C082E69AE00E948D069DCF2F
:1046500090919A0293FBCC27C0F981E0C827892F5B
:10466000C0FB83F980939A02CC2351F086E59AE04F
:104670000E948D0680919A02816080939A0233C0D5
:1046800089E49AE0E2CF0E945A26162F072FF82ECF
:10469000E92ED091D002C0911A010E94D624EF9247
:1046A000FF920F931F931F92DF931F92CF931F923E
:1046B0008F9388ED95E09F938F930E9426078DB787
:1046C0009EB70C960FB6F8949EBF0FBE8DBF5DCF00
:1046D000895301C080E00E94CC2157CF87E49AE043
:1046E0000E948D06C0E08C2FDF91CF911F910F911A
:1046F000FF90EF90089580E008950C947B23CF9372
:10470000C82F8091B402813071F040F0823009F0FE
:1047100045C08C2F0E94AF2081E046C00E94061247
:104720008232F1F504C00E940612823261F48C2FAD
:104730000E947D23811104C08C2F0E94EC212CC08B
:1047400081E090E029C08C2F0E947B23811123C03F
:10475000C431C9F058F4CB3069F0C031B9F482E00B
:104760008093B40288E30E94AF2015C0C93259F08B
:10477000C83361F48FEF96E00E948D068FEC95E0D0
:104780000E948D0608C01092B4020CC08DEC95E01A
:104790000E948D0607C081E0817006C01092B402AD
:1047A00080E002C080E0F8CFCF910895CF93DF93EF
:1047B00086319C4541F5EB010E940612982F8A81B3
:1047C0002091020130910301882379F09A7A81E0E7
:1047D00009F480E08093B502911102C069E201C042
:1047E00065E3C9010E94A7250AC08091B502811125
:1047F00002C069E201C065E3C9010E94A9250E94C7
:10480000481280E001C081E0DF91CF9108950F93BD
:104810001F93CF93DF93C42FD22FFC018281882373
:10482000C9F04093B8020E944E269093B70280933D
:10483000B60280E28C0F883008F057C0C77081E064
:1048400001C0880FCA95EAF7DF91CF911F910F91B0
:104850000C94100A8091B802481330C08091B602BF
:104860009091B7020E946626883C910538F510E2C7
:104870001D0FCD17B9F080E28C0F883040F4C7705F
:1048800081E001C0880FCA95EAF70E94170A183024
:1048900028F581E09D2F977001C0880F9A95EAF75F
:1048A0000E94100A802F0E94070A1830F0F4D77077
:1048B00081E001C0880FDA95EAF70AC080E28C0F28
:1048C000883098F4C77081E001C0880FCA95EAF774
:1048D000DF91CF911F910F910C94170A802FDF91D8
:1048E000CF911F910F910C94070ADF91CF911F91E7
:1048F0000F9108950F939C01CB01243F4CE53407A1
:1049000031F188F4293DFCE53F07D9F02A3D4CE51B
:10491000340779F1283D3C45A9F506E221EE41EE48
:1049200068ED7CE52BC0263FFCE53F07E1F0A8F0F1
:10493000273F3C4539F507E225EE46EE67EF7CE57B
:104940001DC007E225EE45EE69ED7CE517C006E2E5
:1049500021EE40EE64EF7CE511C007E225EE44EE67
:1049600065EF7CE50BC006E221EE42EE66EF7CE5EA
:1049700005C008E221E045EE6AED7CE50E940724CF
:1049800080E008C0FC018281882319F01092B802EF
:1049900001C081E00F9108959093FF018093FE0183
:1049A00008959093BE028093BD020895E091BD02E8
:1049B000F091BE02309721F00190F081E02D099432
:1049C00080E00895EF92FF920F931F93CF93DF93B0
:1049D000E091BD02F091BE023097B1F18C010280EE
:1049E000F381E02D099580919A0282FF2DC080FF0E
:1049F00004C08EEE9AE00E948D06E80118E088EE71
:104A0000E82E8AE0F82E80919A0280FF0BC0888100
:104A10001F928F93FF92EF920E9426070F900F90A4
:104A20000F900F90115021961111EDCF80919A02A5
:104A300080FF0AC086EE9AE0DF91CF911F910F911F
:104A4000FF90EF900C948D06DF91CF911F910F9105
:104A5000FF90EF900895E091BD02F091BE02309773
:104A600039F022E0DC012C930480F581E02D0994DB
:104A700008952091BB023091BC022817390771F0CC
:104A80009093BC028093BB02E091BD02F091BE0204
:104A9000309721F00680F781E02D09940895209148
:104AA000B9023091BA022817390771F09093BA020F
:104AB0008093B902E091BD02F091BE02309721F0DF
:104AC0000084F185E02D09940895FC01329697E069
:104AD00080E0915029F021912223D9F38F5FF9CF03
:104AE0000895662349F0FC013296089621916217D9
:104AF00029F0E817F907D1F780E0089581E00895DB
:104B00009C01FC0132969FEF80E04191461789F0AD
:104B10009F3F19F4411101C0982F8F5F8630A9F78C
:104B20009F3F39F0F901E90FF11D97FDFA95628376
:104B3000089508959C012A5F3F4FFC01428146136E
:104B400001C01282019682179307B9F708950C9459
:104B500080250C949A25029626E0FC0111922A9554
:104B6000E9F7089508950C94B22583E08093BF027D
:104B70000C94B325811102C081E001C082E08093D2
:104B8000BF020C94B3250C94BA2581E08093BF0238
:104B90000C94B3250C94C52508950C94CC250C9445
:104BA000CD250C94CC250C94CC250C94CC25CF93FE
:104BB0000E94D3250E94F9170E94D125C0E08C2FB6
:104BC0000E94DD16892B29F4CF5FC530C1F780E044
:104BD00001C081E0CF91089508951F920F920FB602
:104BE0000F9211248F939F93AF93BF938091C00234
:104BF000811113C08091E8029091E902A091EA022C
:104C0000B091EB024196A11DB11D8093E8029093F3
:104C1000E902A093EA02B093EB02BF91AF919F919A
:104C20008F910F900FBE0F901F9018958091F002FA
:104C3000843031F10E940D081092C00220E488E116
:104C400090E00FB6F894A895809360000FBE209373
:104C5000600083B7817F846083BF83B7816083BF37
:104C60007894889583B78E7F83BF0FB6F894A89504
:104C700080916000886180936000109260000FBE98
:104C800008950E94B30C0C94140882E084BD93E054
:104C900095BD9AEF97BD80936E0008952FB7F89455
:104CA0008091E8029091E902A091EA02B091EB02B2
:104CB0002FBF08952FB7F8946091E8027091E90230
:104CC0008091EA029091EB022FBF08959C014FB7AB
:104CD000F8948091E8029091E902A091EA02B091E3
:104CE000EB024FBF821B930B089578941F920F9293
:104CF0000FB60F9211248F939F93AF93BF93809120
:104D0000E8029091E902A091EA02B091EB020196CB
:104D1000A11DB11D8093E8029093E902A093EA02DD
:104D2000B093EB02BF91AF919F918F910F900FBE07
:104D30000F901F90189581E08093E00080E28093AF
:104D4000D8001092C9008FE19EE40197F1F700C0EE
:104D5000000087E090EBDC018093F9029093FA0267
:104D6000A093FB02B093FC029CE088E10FB6F8949C
:104D7000A895809360000FBE90936000FFCF809154
:104D8000CF020895089522E02093E9002FEF30919B
:104D9000E800215035FD06C035ED3A95F1F70000E9
:104DA0002111F5CF2091E80025FF0BC040E050E035
:104DB00066E070E00E94AB298091E8008E778093D6
:104DC000E8000895CF93DF9321E02093E9002FEFCF
:104DD0003091E800215035FD06C035ED3A95F1F7E8
:104DE00000002111F5CF2091E80025FF14C0EC014F
:104DF00040E050E068E070E00E94AB298091E8005C
:104E00008E778093E80088E0FE01A7ECB2E0019085
:104E10000D928A95E1F7DF91CF9108958093C302B7
:104E20007093C5026093C4028091F002843001F552
:104E300082E08093E9008FEF9091E800815095FD2A
:104E400006C095ED9A95F1F700008111F5CF80919C
:104E5000E80085FF0DC040E050E063E070E083ECC7
:104E600092E00E94AB298091E8008E778093E80061
:104E70000895BC0184E00C940E27BC0183E00C94DF
:104E80000E2784E19BE00E948D068091EF02811144
:104E900009C00E943C2B0E94992B8091E200846003
:104EA0008093E200089580E19BE00E948D061092BD
:104EB000EF0208958CE09BE00E948D060C94CA25B9
:104EC00088E09BE00E948D066091EC0281E0611118
:104ED00001C080E00C94B52584E09BE00E948D0623
:104EE0009091F00281E0943009F080E06091EC0252
:104EF0000C94BA252091C2022F5F822F62E30E9498
:104F0000582E992319F02093C20208951092C202DC
:104F10008091C602882371F18091F002843041F5BE
:104F20008091E9008F702091EC00922F917020FD0C
:104F300090E8892B93E09093E9009091EB0090FF2B
:104F400014C09091EE0097FF10C09091E80095FF7B
:104F500003C01092F100F9CF9091E80090FF05C0D6
:104F60009091E8009E779093E8008F708093E9001D
:104F70001092C602089542E061EC81E00E94B52AD9
:104F800042E261EC82E00E94B52A42E261EC83E0F9
:104F90000E94B52A9091F00281E0943009F080E0FF
:104FA0006091EC020C94C3258091F202833009F4E5
:104FB00061C030F4813071F0823009F49AC00895F4
:104FC0008A3009F486C08B3009F46CC0893009F04E
:104FD000A8C020C08091F102813A09F0A2C080915E
:104FE000E800877F8093E8008091F5029091F602B7
:104FF000892B21F468E087EC92E003C060E080E058
:1050000090E070E00E94F6298091E8008B77809311
:10501000E80008958091F102813209F082C0809108
:10502000F5029091F602029708F07BC08091E800AB
:10503000877F8093E8008091E80082FD05C0809121
:10504000F0028111F8CF6DC02091F3008091F20041
:1050500090E0922B029731F48091F100813011F0B1
:10506000863021F48091F1008093CF028091E80096
:105070008B7753C08091F102813A09F052C0809140
:10508000F5029091F602892B09F04BC08091E8005F
:10509000877F8093E8008091E80080FFFCCF8091BB
:1050A0001A0136C08091F1028132D9F58091F50262
:1050B0009091F602892BA9F58091E800877F809373
:1050C000E8000E94EA2A8091F30280931A010C946E
:1050D000B30C8091F102813221F58091E800877F45
:1050E0008093E8000E94EA2A8091F4028093D00223
:1050F00008958091F102813AA1F48091E800877FC0
:105100008093E8008091E80080FFFCCF8091D0027E
:105110008093F1008091E8008E778093E8000C94F2
:10512000EA2A08959FB7F8941092C6029FBF909103
:10513000F002943009F057C09091E9009F703091CF
:10514000EC00232F217030FD20E8922B23E02093E8
:10515000E9002091EB0020FF43C02091EE0027FFE3
:105160003FC02091C102222321F02091E80025FFB9
:1051700037C01092C10226E03091E80035FD15C01D
:105180003091F002343061F53091EB0035FD28C0EC
:10519000215021F481E08093C10222C0EFE9FFE0B9
:1051A0003197F1F700C00000E7CF8093F1008091C4
:1051B000E80085FD0AC08091E80080FFFCCF809167
:1051C000E8008E778093E80006C08FB7F89421E05E
:1051D0002093C6028FBF9F709093E90080E00895EE
:1051E0009F709093E9008FEF089584B7877F84BF05
:1051F0000FB6F894A8958091600088618093600054
:10520000109260000FBE90E080E80FB6F894809393
:105210006100909361000FBE0C94C5250E943C2B49
:105220000E94992BE2EEF0E0808184608083789484
:105230000C942D2E8EE091E00C94D1248091F002FC
:105240008530C9F480E09BE00E948D068091F002D9
:10525000853079F40E9416268091EE028823B1F3FE
:105260000E94D725882391F30E9495290E94B30CB0
:10527000EDCF0C944126089508950C943F29292FD1
:10528000332723303105C9F060F42130310581F036
:105290002230310509F041C08BE590E024E43BE089
:1052A00040C021323105E1F02232310531F135C003
:1052B00082E190E02FE93BE034C0992781309105ED
:1052C00049F028F0029749F5E8E1FBE005C0E0E489
:1052D000FBE002C0E6E2FBE0849190E09F0121C088
:1052E00063307105D0F4660F771FFB01E850FE4F65
:1052F0002081318189E090E014C06330710568F449
:10530000FB01EE0FFF1FEE50FE4F20813181FB01AC
:10531000E151FE4F808190E004C080E090E020E009
:1053200030E0FA0131832083089580E189BD82E174
:1053300089BD09B400FEFDCF8091D8008F7D809398
:10534000D8008091E00082608093E0008091E000CE
:1053500081FDFCCF0895CF92DF92EF92FF920F93E1
:105360001F93CF93DF93EC018B017A010E94092BED
:10537000811133C0E114F10439F0F701808191818A
:10538000081B190BC80FD91FC12CD12C01151105F1
:1053900019F18091E80085FD16C08091E8008E77B4
:1053A0008093E800E114F10449F0F70180819181D4
:1053B000C80ED91ED182C08285E00FC00E94092B81
:1053C000882321F30AC089918093F10001501109CB
:1053D000FFEFCF1ADF0ADACF80E0DF91CF911F9184
:1053E0000F91FF90EF90DF90CF9008952091F702FA
:1053F0003091F8022617370748F06115710539F426
:105400002091E8002E772093E80001C0B901FC014B
:1054100020E06115710579F18091F0028823F1F1A6
:105420008530F1F18091E80083FD3CC08091E80077
:1054300082FD2EC08091E80080FFEBCF2091F30029
:105440008091F20090E0922B6115710551F0883047
:10545000910538F421912093F10061507109019672
:10546000F3CF21E0089709F020E08091E8008E77E3
:105470008093E800CECF2111CFCF0AC08091F002F7
:10548000882361F0853061F08091E80083FD0AC0D7
:105490008091E80082FFF2CF80E0089582E00895D5
:1054A00083E0089581E008952091F7023091F80299
:1054B0002617370748F06115710539F42091E80087
:1054C0002E772093E80001C0B901FC0120E06115AE
:1054D000710591F18091F002882309F440C0853074
:1054E00009F43FC08091E80083FD3DC08091E80051
:1054F00082FD2FC08091E80080FFE9CF2091F3006A
:105500008091F20090E0922B6115710559F088307E
:10551000910540F424912093F10031966150710976
:105520000196F2CF21E0089709F020E08091E80091
:105530008E778093E800CBCF2111CCCF0AC0809129
:10554000F002882361F0853061F08091E80083FDEE
:105550000AC08091E80082FFF2CF80E0089582E0E7
:10556000089583E0089581E00895982F973068F5B5
:105570009093E900981739F07091EC002091ED00BC
:105580005091F00003C0242F762F50E021FD02C07F
:105590009F5FECCF3091EB003E7F3093EB0030917A
:1055A000ED003D7F3093ED003091EB0031603093A2
:1055B000EB007093EC002093ED005093F0002091ED
:1055C000EE0027FDE5CF80E008958F708093E9001D
:1055D00081E008958091F10287FF11C08091E80079
:1055E00082FD05C08091F0028111F8CF11C0809139
:1055F000E8008B770BC08091F002882349F08091FE
:10560000E80080FFF8CF8091E8008E778093E80073
:1056100008952091E4003091E50095E64091EC007A
:10562000842F817040FF23C08091E80080FD1DC061
:105630008091F002882399F0853099F08091EB00F9
:1056400085FD11C04091E4005091E5002417350715
:1056500029F3915011F09A01E1CF84E0089582E09E
:10566000089583E0089581E0089580E008954091D1
:10567000E80042FFDDCF08950E94AA2B0E94B22BC2
:10568000E0EEF0E0808181608083E8EDF0E08081F1
:105690008F77808319BCA7EDB0E08C918E7F8C93BF
:1056A00080818F7E80831092EF0208950F931F9365
:1056B000CF93DF930E94AA2B0E94B22BC8EDD0E0BB
:1056C00088818F77888388818068888388818F7DAF
:1056D000888319BC1092F0021092EC021092EE0234
:1056E0001092ED0200EE10E0F80180818B7F808344
:1056F00088818160888342E060E080E00E94B52A72
:10570000E1EEF0E080818E7F8083E2EEF0E0808148
:1057100081608083808188608083F80180818E7FB2
:105720008083888180618883DF91CF911F910F9161
:105730000895E8EDF0E080818F7E8083E7EDF0E072
:1057400080818160808384E082BF81E08093EF026A
:105750000C94562BE8EDF0E080818E7F80831092D0
:10576000E20008951092DA001092E10008951F926D
:105770000F920FB60F9211242F933F934F935F9385
:105780006F937F938F939F93AF93BF93EF93FF9309
:105790008091E10082FF0BC08091E20082FF07C090
:1057A0008091E1008B7F8093E1000E947A278091B5
:1057B000DA0080FF1FC08091D80080FF1BC080915D
:1057C000DA008E7F8093DA008091D90080FF0DC0CF
:1057D00080E189BD82E189BD09B400FEFDCF81E091
:1057E0008093F0020E94412705C019BC1092F0027C
:1057F0000E9453278091E10080FF19C08091E20050
:1058000080FF15C08091E2008E7F8093E20080913E
:10581000E20080618093E2008091D80080628093F2
:10582000D80019BC85E08093F0020E946027809127
:10583000E10084FF30C08091E20084FF2CC080E151
:1058400089BD82E189BD09B400FEFDCF8091D800F9
:105850008F7D8093D8008091E1008F7E8093E1005E
:105860008091E2008F7E8093E2008091E20081606F
:105870008093E2008091EC02882311F084E007C05D
:105880008091E30087FD02C081E001C083E0809346
:10589000F0020E946C278091E10083FF29C0809173
:1058A000E20083FF25C08091E100877F8093E100C3
:1058B00082E08093F0021092EC028091E1008E7FF2
:1058C0008093E1008091E2008E7F8093E2008091DE
:1058D000E20080618093E20042E060E080E00E94AC
:1058E000B52A8091F00088608093F0000E945A27CA
:1058F000FF91EF91BF91AF919F918F917F916F91A8
:105900005F914F913F912F910F900FBE0F901F907D
:1059100018951F920F920FB60F9211242F933F9359
:105920004F935F936F937F938F939F93AF93BF93A7
:10593000CF93DF93EF93FF93C091E900CF708091F5
:10594000EC00D82FD17080FDD0E81092E900809152
:10595000F000877F8093F00078940E94CD2C109205
:10596000E9008091F00088608093F000CD2BCF702B
:10597000C093E900FF91EF91DF91CF91BF91AF917B
:105980009F918F917F916F915F914F913F912F9157
:105990000F900FBE0F901F9018951F93CF93DF931A
:1059A000CDB7DEB7AA970FB6F894DEBF0FBECDBF56
:1059B000E1EFF2E08091F100819322E0E93FF2070C
:1059C000C9F70E94D4278091E80083FF2EC18091FF
:1059D000F1029091F202492F50E04A30510508F04F
:1059E00024C1FA01E759FF4F0C94AE2E803821F004
:1059F000823809F01AC108C08091ED029091EE0240
:105A0000992389F082600FC08091F5028F708730F2
:105A100008F00BC18093E9008091EB0085FB88279B
:105A200080F91092E9009091E800977F9093E80048
:105A30008093F1001092F100D1C0282F2D7F09F042
:105A4000F4C0882319F0823061F0EFC08091F30236
:105A5000813009F0EAC0933009F080E08093EE02D3
:105A60002EC08091F30281112AC08091F5028F70BF
:105A70002FEF280F263008F0D8C08093E90020913E
:105A8000EB0020FF1CC0933021F48091EB0080627A
:105A900014C09091EB0090619093EB0021E030E016
:105AA000A90102C0440F551F8A95E2F74093EA000E
:105AB0001092EA008091EB0088608093EB001092D6
:105AC000E9008091E800877F8093E8000E94EA2A3D
:105AD000ACC08111AAC01091F3021F778091E3003E
:105AE0008078812B8093E3008091E800877F80930A
:105AF000E8000E94EA2A8091E80080FFFCCF8091B4
:105B0000E30080688093E300111102C082E001C0CD
:105B100083E08093F00289C08058823008F085C00D
:105B20008091F3029091F4028C3D53E0950779F552
:105B300083E08A838AE289834FB7F894DE01139663
:105B400020E03EE051E2E32FF0E050935700E49173
:105B500020FF03C0E295EF703F5FEF708E2F90E063
:105B6000EA3010F0C79601C0C0968D939D932F5FC9
:105B7000243149F74FBF8091E800877F8093E80088
:105B80006AE270E0CE0101960E94F62916C060918B
:105B9000F5027091F602AE014F5F5F4F0E943D2902
:105BA000BC01892B09F441C09091E800977F909344
:105BB000E80089819A810E94542A8091E8008B77BD
:105BC0008093E80032C0803881F58091E800877FBB
:105BD0008093E8008091EC028093F1008091E800CE
:105BE0008E7772CF811121C08091F3029091F402DF
:105BF00099270297D4F48091E800877F8093E8008A
:105C00008091F3028093EC020E94EA2A8091EC02D8
:105C1000811106C08091E30087FD02C081E001C0D0
:105C200084E08093F0020E94BB278091E80083FF0C
:105C30000AC08091E800877F8093E8008091EB00A4
:105C400080628093EB00AA960FB6F894DEBF0FBE79
:105C5000CDBFDF91CF911F910895CF938091F00236
:105C60008823A1F0C091E900CF709091EC00892FBA
:105C7000817090FD80E8C82B1092E9008091E800C7
:105C800083FD0E94CD2CCF70C093E900CF91089581
:105C9000DB018F939F930E94C32EBF91AF91A29F70
:105CA000800D911DA39F900DB29F900D112408951A
:105CB000991B79E004C0991F961708F0961B881F5E
:105CC0007A95C9F780950895AA1BBB1B51E107C0BF
:105CD000AA1FBB1FA617B70710F0A61BB70B881F7C
:105CE000991F5A95A9F780959095BC01CD0108950B
:105CF00097FB072E16F4009407D077FD09D00E9479
:105D0000642E07FC05D03EF4909581959F4F089531
:105D1000709561957F4F0895A1E21A2EAA1BBB1BB7
:105D2000FD010DC0AA1FBB1FEE1FFF1FA217B30767
:105D3000E407F50720F0A21BB30BE40BF50B661F7D
:105D4000771F881F991F1A9469F760957095809541
:105D500090959B01AC01BD01CF010895EE0FFF1F8F
:105D60000590F491E02D0994A29FB001B39FC0016A
:105D7000A39F700D811D1124911DB29F700D811D77
:105D80001124911D08950E94B42EA59F900DB49FDB
:105D9000900DA49F800D911D11240895FB01DC013D
:105DA00004C08D910190801921F441505040C8F7F2
:105DB000881B990B0895F999FECF92BD81BDF89A81
:105DC000992780B50895A8E1B0E042E050E00C9436
:105DD0000F2F262FF999FECF92BD81BDF89A01971A
:105DE00000B4021639F01FBA20BD0FB6F894FA9A23
:105DF000F99A0FBE08950396272F0E94EA2E0E945B
:105E0000E92E252F0E94EA2E242F0C94EA2E0196CB
:105E1000272F0E94EA2E0C94E92EDC01CB01FC0115
:105E2000F999FECF06C0F2BDE1BDF89A319600B4F3
:0E5E30000D9241505040B8F70895F894FFCFFE
:105E3E00C8007E02280850011E0A14010601BF2662
:105E4E00E226C3263D273927C22601E200E900EAF1
:105E5E0000B500B600B700CD008301CC008A0192D8
:105E6E000194012102230224022502260227022A7E
:105E7E0002B300B4006F007000818283E200E9007B
:105E8E00EA00B500B600B700CD008301CC008A0150
:105E9E0092019401210223022402250226022702E6
:105EAE002A02B300B4006F007000818283F0333297
:105EBE0031303790919293959697343536F7F6F5B3
:105ECE00F4F13F3F3F006D6B5F64656C6179006D6F
:105EDE006B5F696E74657276616C006D6B5F6D6180
:105EEE00785F7370656564006D6B5F74696D655F77
:105EFE00746F5F6D6178006D6B5F776865656C5F61
:105F0E006D61785F7370656564006D6B5F77686552
:105F1E00656C5F74696D655F746F5F6D617800406D
:0E5F2E007B224E0CD30BB10B560B6F0B880B66
:00000001FF
